:100000000000022049430008BD2D0008C12D000852
:10001000C52D0008C92D0008CD2D000800000000E6
:10002000000000000000000000000000D12D0008CA
:10003000D52D000800000000D92D0008DD2D000896
:100040009943000899430008994300089943000820
:100050009943000899430008994300089943000810
:100060009943000899430008994300089943000800
:1000700099430008994300089943000899430008F0
:1000800099430008994300089943000899430008E0
:1000900099430008994300089943000899430008D0
:1000A00099430008994300089943000899430008C0
:1000B00099430008994300089943000899430008B0
:1000C00099430008994300089943000899430008A0
:1000D00099430008E52D0008F52D00089943000814
:1000E0009943000899430008994300089943000880
:1000F0009943000899430008994300089943000870
:10010000994300089943000899430008994300085F
:10011000052E0008994300089943000899430008F8
:10012000994300089943000899430008994300083F
:10013000994300089943000899430008994300082F
:10014000994300089943000899430008994300081F
:10015000994300089943000899430008994300080F
:1001600099430008994300089943000899430008FF
:1001700099430008994300089943000800000000D3
:080180009943000899430008AF
:10019000044B05481B1A062B02D9044B03B1184720
:1001A000704700BF7F0000207C000020000000009E
:1001B00005490648091A891001EBD171491002D08E
:1001C000034B03B1184770477C0000207C000020DF
:1001D0000000000010B5064C237843B9FFF7D8FFA4
:1001E000044B13B10448AFF300800123237010BD0A
:1001F0007C000020000000009C43000808B5084B6C
:100200001BB108490848AFF300800848036813B9D8
:10021000BDE80840CCE7064B002BF9D09847F7E73C
:1002200000000000800000209C4300087C000020AB
:100230000000000070B50F4E0F4D761BB61018BFB2
:10024000002405D0013455F8043B9847A642F9D163
:100250000A4E0B4D761B04F0A1F8B61018BF00240F
:1002600006D0013455F8043B9847A642F9D170BD39
:1002700070BD00BFCC440008CC440008D044000846
:10028000CC44000870B4840746D0541E002A41D0E4
:10029000CDB2034602E0621EE4B3144603F8015BEC
:1002A0009A07F8D1032C2ED9CDB245EA05250F2C9B
:1002B00045EA054519D903F110022646103E0F2ED6
:1002C00042F8105C42F80C5C42F8085C42F8045CAE
:1002D00002F11002F2D8A4F1100222F00F0204F091
:1002E0000F041032032C13440DD91E462246043A43
:1002F000032A46F8045BFAD8221F22F003020432D4
:10030000134404F003042CB1C9B21C4403F8011BCC
:10031000A342FBD170BC704714460346C2E700BF3E
:100320000EB410B5044683B018B183690BB900F060
:100330004DFB06A803460190059AA168204600F0EF
:1003400009FD03B0BDE8104003B070470FB410B50D
:100350000A4B1C6882B024B1A36913B9204600F08F
:1003600035FB05A803460190049AA168204600F0D9
:10037000F1FC02B0BDE8104004B07047000000205E
:100380002DE9F0410E46804600283ED08369002BBF
:1003900039D084682F4B9C4243D02F4B9C4256D07F
:1003A0002E4B9C4208BFD8F80C40A3891B073DD5B3
:1003B0002369002B3AD0013EA36816F8015F013B88
:1003C000A360B5B1002B04DB23685A1C22601D70AA
:1003D000F2E7A769BB4222462946404601DB0A2DC7
:1003E000F2D100F045F80130E6D14FF0FF30BDE822
:1003F000F081002B21DB23680A22591C21601A702E
:100400001046BDE8F08100F0E1FAD8F81830D8F8CD
:100410000840002BBED1404600F0D8FA0D4B9C425C
:10042000BBD1D8F80440A3891B07C1D4214640465C
:1004300000F080F80028BED0D7E7224640460A21C7
:1004400000F016F80130D0D00A20BDE8F081D8F8CD
:100450000840AAE7F8430008D8430008B84300085A
:10046000024B01461868FFF78BBF00BF0000002059
:10047000F8B50E461446054610B18369002B41D0ED
:10048000254B9C4243D0254B9C4242D0244B9C425E
:1004900008BFEC68A389A269A2601A0721D5236965
:1004A000FBB122686169D31A8B42F7B221DA0133BA
:1004B000A168501C0139A1602060167062699A42DF
:1004C00006D0A389DB0701D50A2F01D03846F8BD35
:1004D0002146284600F040F90028F7D04FF0FF37BA
:1004E000F4E72146284600F025F80028F6D12369D4
:1004F000D7E72146284600F02FF90028EED12268E0
:100500000123D5E700F062FA034B9C42BBD16C6833
:10051000C0E7AC68BEE700BFF8430008D843000856
:10052000B8430008024B0A4601461868FFF7A0BF0F
:1005300000000020384B70B51D6806460C4615B10A
:10054000AB69002B42D0354B9C4245D0344B9C428A
:1005500058D0344B9C4208BFEC68B4F90C2093B2DD
:1005600019070CD52069A8B113F001021ED06369E8
:1005700000225B42A361A260F0B1002070BDDD06E5
:1005800042D558072AD4206942F00803A3819BB2C0
:100590000028E9D103F42072B2F5007FE4D03046A0
:1005A000214600F0B1FAA3892069DDE7990758BF19
:1005B0006269A2600028E0D1B4F90C301A06DDD5DA
:1005C00043F04003A3814FF0FF3070BD284600F098
:1005D000FDF9124B9C42B9D16C68BEE7616B51B119
:1005E00004F14403994204D0304600F0D1FAB4F942
:1005F0000C200023636300232069636022F024023F
:100600002060C1E7AC68A8E742F0400209233360EC
:100610004FF0FF30A28170BD00000020F8430008B9
:10062000D8430008B84300088B891A072DE9F04128
:100630000D46804635D44A68002A6BDDEC6A002CF2
:1006400047D003F48052002192B2D8F80060C8F875
:100650000010002A62D06A6D5F0705D569686B6B70
:10066000521A0BB12B6CD21A0023296A4046A047BC
:10067000441C39D0AB892A692A60DB044FF00002A0
:100680006A6045D4696BC8F8006011B305F1440392
:10069000994202D0404600F07BFA00206863BDE832
:1006A000F0810E69AEB10C680E6098070CBF4B6903
:1006B0000023A41B8B600AE023463246AF6A296AF6
:1006C0004046B8470028A4EB0004064404DD002C93
:1006D000F2DC0020BDE8F081AB8943F04003AB8140
:1006E0004FF0FF30BDE8F081D8F800201D2AF3D884
:1006F000184BD34003F0010383F00101002BEBD032
:10070000AB892C696960D9042C60BBD5002AB9D1AA
:100710006865B7E70A6C002A90DCDAE70123296AEA
:100720004046A047431C024602D0AB89EC6A93E7DF
:10073000D8F80030002BF8D01D2B01D0162B02D199
:10074000C8F80060C5E7AB8943F04003AB81BDE862
:10075000F08100BF010040200B6933B310B504469F
:1007600082B008B18369ABB1114B994219D0114BDA
:10077000994218D0104B994208BFE168B1F90C308A
:1007800013B9002002B010BD204602B0BDE81040F1
:10079000FFF74ABF019100F019F90199044B994202
:1007A000E5D16168EAE7A168E8E70020704700BF8B
:1007B000F8430008D8430008B843000820B1054BAF
:1007C00001461868FFF7C8BF034B0449186800F0DA
:1007D00043B900BF00000020B443000859070008D7
:1007E00000207047014900F037B900BF59070008E1
:1007F0000020704770B568234D1E03FB05F50E46BB
:1008000005F1740100F00AFA044640B100210C30F1
:10081000666005F168022160A060FFF733FD2046A5
:1008200070BD00BF1F4B70B51D68AB69064613B99C
:10083000284600F039F848356B68AC68013B05D5AF
:1008400021E0013B5A1C04F168041CD0B4F90C20CF
:10085000002AF6D1002501234FF6FF72E281A38121
:1008600065662560A560656025616561A5612946AD
:10087000082204F15C00FFF705FD6563A563A5642C
:10088000E564204670BD2B680BB11D46D4E70421FA
:100890003046FFF7AFFF286008B10546CCE70C23D0
:1008A000336070BDB44300083D4B3E491A682DE9E2
:1008B000F04F90424FF000038364C364036508BFA8
:1008C000012383B008BF836181620746FFF7AAFF57
:1008D00078603846FFF7A6FFB8603846FFF7A2FFFA
:1008E0007D68F86000240423AB812C606C60AC60F0
:1008F0006C66EC812C616C61AC61214605F15C0099
:100900000822FFF7BFFCBE68DFF89CB0DFF89CA0B0
:10091000DFF89C90DFF89C80C5F824B00123092201
:10092000C5F828A0C5F82C90C5F830802D62214666
:10093000F381B28134607460B46074663461746150
:10094000B46106F15C0008220193FFF79BFCFD688F
:10095000366212200222C6F824B0C6F828A0C6F8D3
:100960002C90C6F830802146A881EA812C606C600A
:10097000AC606C662C616C61AC6105F15C000822B6
:10098000FFF780FC019B2D62C5F824B0C5F828A0B4
:10099000C5F82C90C5F83080BB6103B0BDE8F08F7E
:1009A000B4430008E5070008D1130008F913000854
:1009B0003514000855140008024B0349186800F06C
:1009C0004BB800BFB443000859070008836903B956
:1009D0006AE77047704700BF704700BF704700BFAD
:1009E000704700BF024B0349186800F00FB800BF02
:1009F00000000020F1070008024B0349186800F0CE
:100A000005B800BF00000020E10700082DE9F04113
:100A100010F148071BD0884600267D68BC68013D60
:100A20000FD4A389012B05F1FF3506D9B4F90E3097
:100A30000133204601D0C04706436B1C04F1680413
:100A4000EFD13F68002FE8D13046BDE8F0813E4647
:100A50003046BDE8F08100BF2DE9F84310F14807AA
:100A60001FD0884606464FF000097D68BC68013DEE
:100A700011D4A389012B05F1FF3508D9B4F90E3043
:100A800001332146304602D0C04749EA00096B1CB9
:100A900004F16804EDD13F68002FE6D14846BDE877
:100AA000F883B9464846BDE8F88300BF70B50C46E8
:100AB000B1F90E10002990B015461E4613DB01AAAD
:100AC00000F0F4FC00280EDB029A02F47042A2F55A
:100AD0000052B2FA82F252094FF480630020326071
:100AE0002B6010B070BDA38900221B06326004D5B4
:100AF000402300202B6010B070BD4FF480630020B5
:100B00002B6010B070BD00BF8A8992070B4606D5D6
:100B100001F1470201211A601A6159617047F0B56D
:100B200083B001AB6A460C460546FFF7BFFF00994C
:100B30000646284600F072F8B4F90C30D0B1019A9C
:100B4000124F0099AF6243F08003A38120602061BF
:100B500061611AB93343A38103B0F0BD2846B4F9EB
:100B60000E1000F039FEB4F90C300028F2D043F03A
:100B70000103EFE79A05EFD404F1470243F00203C3
:100B80000121A381226022616161E5E7E507000898
:100B900030B481B151F8043C0439002BB8BFC918F6
:100BA0001D4B1A682AB18A420AD908680C18A24259
:100BB00025D04A60196030BC70478B4203D81A4672
:100BC0005368002BF9D1146815198D420CD007D841
:100BD00008680C189C4218D04B6030BC51607047BC
:100BE0000C23036030BC704709680C44111999420A
:100BF0001460E0D10ACB0C4453601460DBE7146846
:100C000052684A6020440860D4E71C685B684B6007
:100C1000204408605160CEE79800002070B5CD1CDC
:100C200025F0030508350C2D38BF0C25002D064690
:100C30003BDBA94239D827490A6852B113685B1BCC
:100C400004D436E023685B1B1AD522465468002C76
:100C5000F8D149681F4C002936D02946304600F0AB
:100C6000A5FB431C21D0C41C24F00304A04205D0E2
:100C7000211A304600F09AFB013016D0256004E0BE
:100C80000B2B0DD923601C44256004F10B0020F0D0
:100C90000700231DC31A02D05A42E25070BD70BD36
:100CA00094420ED063685360EFE70C23336000205A
:100CB00070BD0B2B03D8536814460B60E5E7144650
:100CC000E0E713461446F8E7304600F06FFB60603B
:100CD000C3E700BF980000209368013B002B10B4CD
:100CE000936008DBCCB21368581C10601970204662
:100CF0005DF8044B70479469A34202DBCCB20A2C26
:100D0000F1D15DF8044BFFF7B3BB00BF93B1F8B569
:100D100014460F460646D51801E0AC4208D03A46C4
:100D200014F8011B3046FFF7D7FF431CF5D1F8BD7F
:100D30000020F8BD00207047936810B5144613B921
:100D40005360184610BD00F0C5FB0023A36063602C
:100D500010BD00BF2DE9F04F9DB0884614460393A7
:100D6000814618B18369002B00F00B818B4B9845AD
:100D700000F00D818A4B984500F00C81894B984515
:100D800008BFD9F80C80B8F80C301D0740F1EF808F
:100D9000D8F81030002B00F0EA8030238DF82A308C
:100DA0002378814DDFF804A20021202209918DF8DB
:100DB0002920002B00F08580252B264603D117E043
:100DC000252B00F0868016F8013F002BF8D1B6EBFA
:100DD000040B76D022465B4641464846FFF796FF15
:100DE00001306ED0099B32785B440993002A68D0A9
:100DF00000234FF0FF31721C0493079306938DF884
:100E000053301A930591012604E0049906FA03F37E
:100E10000B430493144664482178052200F008FD32
:100E2000621C431B0028F0D1049BD80644BF20223B
:100E30008DF853201907217844BF2B228DF85320B9
:100E40002A2968D0A1F13002092A0BD8079B14F88F
:100E5000011F03EB830302EB4303A1F13002092AD4
:100E6000F5D907932E293FD00322504800F0E0FC2B
:100E700048B10499CAEB0000402202FA00F041EAAE
:100E8000000301340493217849488DF82810062284
:100E9000013400F0CDFC00285FD0464BEBB103AB32
:100EA00000934246444B04A94846AFF300800746EE
:100EB0007A1C06D0099B3B4409932378002B7FF4CE
:100EC0007BAFB8F80C305B0658D409981DB0BDE86C
:100ED000F08FB6EB040B8BD07CE7039B073323F03A
:100EE000070308330393E5E761782A291DD0A1F1B0
:100EF00030020023092A04F101040593B4D814F840
:100F0000011F03EB830302EB4303A1F13002092A23
:100F1000F5D90593A8E7039A1168043200290392D2
:100F200015DB0791617801349CE7039B1A680592F1
:100F3000002A03F104030393B8BF4FF0FF3204F11A
:100F40000203AEBFA178A17805921C468CE7494206
:100F500043F0020307910493E4E703AB0093424696
:100F6000154B04A9484600F0CDF80746A0E74146D6
:100F70004846FFF7DFFA00283FF40FAF4FF0FF308D
:100F8000A4E7FFF723FD054B98457FF4F3AED9F8AE
:100F90000480F8E6D9F80880F5E600BFF8430008B9
:100FA000D8430008B843000888440008904400086B
:100FB00094440008000000000D0D000810B4044C1B
:100FC00013460A46014620685DF8044BFFF7C2BE8F
:100FD000000000202DE9F0470C4691460969A268FF
:100FE000DDF820808A42B8BF0A46C9F8002094F88C
:100FF000431006461F4611B10132C9F8002023688C
:1010000099065DD5D9F800200232C9F8002023687E
:1010100013F0060F19461DD1E1688A1A002AD8BFBD
:10102000194617DD04F1190A002505E0E368D9F82F
:1010300000209B1AAB420CDD012352463946304654
:10104000C047013005F10105F0D14FF0FF30BDE898
:10105000F087216894F84330003318BF01238A06D3
:101060000AD5E1185A1C302081F84300224494F834
:10107000451082F84310023304F1430239463046EA
:10108000C0470130E1D0236803F00603042B29D0C8
:10109000A36822699342C8BF4FF000092FDD9B1A55
:1010A00099441A34002501E04D4528D001232246F9
:1010B00039463046C047013005F10105F4D1C4E797
:1010C00013F0060F08D1E168D9F800208A1A002A27
:1010D000D8BF1946A6DCBDE794F84330003318BFEB
:1010E0000123C9E7D9F80000E168A3682269091A59
:1010F000934221EAE179D2DCB9F1000FD1D100208D
:10110000BDE8F0872DE9F0430C46097E85B06E29D5
:10111000064617460C98984604F1430C5AD01AD844
:10112000632900F0128100F2D68000295CD0582992
:1011300040F0F58084F8451022680368DFF864E227
:10114000150603F104011ED4550653BF1B68016048
:101150001B88016019E0732900F0CF807ED86F29C9
:1011600000F0E480702940F0DA80226842F020022A
:101170002260782384F845300368DFF82CE21506F6
:1011800003F10401E0D51B680160D00744BF42F0C1
:1011900020022260002B40F09080226822F0200282
:1011A00022601021002284F843206068A06000289B
:1011B000C0F28880226822F004022260002B62D1F3
:1011C000002840F08180654608296AD0C5EB0C03F1
:1011D00023610CE023681A0640F1D5800368626938
:1011E000191D01601B681A60002365462361CDF854
:1011F00000803B4603AA21463046FFF7EBFE013054
:1012000021D02A46236939463046C04701301AD0DA
:101210002368039813F0020FE36819D01A1A002A02
:1012200016DD04F11909002504E0E36803981A1A91
:10123000AA420DDD01234A4639463046C0470130F7
:1012400005F10105F1D14FF0FF3005B0BDE8F083A5
:101250009842B8BF184605B0BDE8F083752965D03F
:1012600078295CD1226884E76168A1602D2000297B
:10127000C3F1000384F8430021DB22F00402DFF80D
:1012800024E122600A216546B3FBF1F201FB123032
:1012900013461EF8002005F8012D002BF4D1082973
:1012A00094D12368D90791D5626823699A428DDC6D
:1012B000302305F8013C013D88E7102172E7DFF893
:1012C000E4E00A21002BDED19EF8003084F84230A1
:1012D00004F1420578E7642901D069291FD1226809
:1012E0000368150603F104013AD51B680160002B61
:1012F000BADBDFF8B0E00A2157E703686268191D1E
:1013000001601D680021284600F092FA002846D0AE
:10131000401B60602061002384F8433067E70123AD
:1013200084F84210236104F14205F4E723681A06A9
:101330001ED503681A1D1B680260227EDFF864E078
:101340006F2A14BF0A2108212CE703681A68191DA7
:101350000123016004F1420584F842202361DAE7A9
:10136000550653BF1B680160B3F900300160BEE74A
:1013700013F0400F036803F1040215BF02601B68FD
:101380001B880260D9E713F0400F0368626903F11C
:10139000040101601B6814BF1A801A6024E76068AA
:1013A000B8E700BF9C440008B044000838B5074CBB
:1013B000002305460846236000F0F4FB431C00D0E0
:1013C00038BD2368002BFBD02B6038BDBC0100204A
:1013D00010B50C46B1F90E1000F09CFB002803DBA1
:1013E000636D0344636510BDA38923F48053A38117
:1013F00010BD00BF002070472DE9F0411646B1F93D
:101400000C201F46D3050C46054607D500220223B3
:10141000B1F90E1000F0F2F9B4F90C20B4F90E1085
:1014200022F48052A2813B4632462846BDE8F04174
:1014300000F014B810B50C46B1F90E1000F0DEF94A
:10144000A389421C0EBF23F4805343F4805360658C
:10145000A38110BDB1F90E1000F016B870B50D469D
:10146000084C114606461A4628460023236000F021
:10147000A7FB431C00D070BD2368002BFBD033605A
:1014800070BD00BFBC01002038B5074C00230546E5
:101490000846236000F05EFB431C00D038BD236883
:1014A000002BFBD02B6038BDBC01002038B50B46AB
:1014B000074C0546114618460023236000F052FBF6
:1014C000431C00D038BD2368002BFBD02B6038BDF7
:1014D000BC0100209368002B76D02DE9F04F8B895A
:1014E00085B00C4619070190164629D522693AB3F2
:1014F00003F002081FFA88F0356800282FD04FF05B
:101500000009B44FC846B246B84543464A4628BFCC
:101510003B460198B8F1000F50D0216AA66AB04747
:10152000002871DDDAF808301B1A8144C0EB080886
:10153000CAF80830002BE7D1002005B0BDE8F08FD5
:1015400021460198FEF7F6FF002840F03A81A38972
:10155000356803F002081FFA88F00028CFD113F095
:1015600001095BD14F4602961FB39A05D4F8088053
:101570002CD54745C246C0F0A48013F4906F40F0CC
:10158000B18020685246494600F03CFAA0682368C2
:10159000C8EB00005344A06023603846029A936869
:1015A0001B1A81443F1A9360002BC5D0A389002FDA
:1015B000DBD1D5F800906F680835D5E7D5F80090F5
:1015C000D5F8048008359FE700207047206823691C
:1015D000984203D861698F4280F0B780B84528BF30
:1015E000B8464246494600F00DFAA3682268C8EBA7
:1015F00003034244A3602260002B49D12146019895
:10160000FFF7AAF8002843D0B4F90C3043F04003A8
:101610004FF0FF30A38105B0BDE8F08F8046029007
:1016200082468146B9F1000F2AD0029B002B4CD094
:10163000206823696269C845C34628BFCB469842E3
:101640005F4604D9A36813449B4500F390809345FB
:1016500020DB1346A76A216A01985246B847071E45
:10166000D2DDB8EB070823D0B368DB1BBA44C7EB65
:101670000909B360002B3FF45FAFB9F1000FD4D17B
:101680000023D5F800A0D5F8049002930835C9E7E7
:10169000404683E75A46514600F0B4F9A2682368F1
:1016A000CBEB02025B44B8EB0708A2602360DBD1FE
:1016B00021460198FFF750F80028A5D1CDF8088001
:1016C000D2E72068B846BA465CE74A460A21504647
:1016D00000F0AEF800286FD001300123CAEB0008FB
:1016E0000293A5E762692068216902EB4208C1EB19
:1016F000000A08EBD8780AF101004FEA680838447C
:101700004045424684BF804642465B0542D511466D
:101710000198FFF783FA8346002855D05246216985
:1017200000F0D6F8A38923F4906343F08003A381EB
:10173000CAEB08030BEB0A00C4F81480C4F810B01D
:101740002060A360B846BA461CE76FF00043BB4276
:1017500028BF3B464A4693FBF1F30198A66A01FB7A
:1017600003F3216AB04700283FF718AF4CE71A4649
:101770005146039300F046F92268039B01981A44EE
:1017800022602146FEF7E8FF039B00287FF43CAF70
:101790001F4666E7019800F099F983460028C7D1F3
:1017A000019D21692846FFF7F3F9B4F90C300C22AA
:1017B00023F080032A6029E7012309F1010802933D
:1017C00036E74FF0FF30B8E6019A0C231360B4F906
:1017D0000C301BE700FCFF7F38B5074C00230546A3
:1017E0000846236000F0C6F9431C00D038BD2368CA
:1017F000002BFBD02B6038BDBC01002070B50D461E
:10180000084C114606461A4628460023236000F07D
:10181000B9F9431C00D070BD2368002BFBD03360A6
:1018200070BD00BFBC0100200000000000000000EF
:1018300001F0FF01102A2BDB10F0070F08D010F881
:10184000013B013A8B422DD010F0070F42B3F6D185
:10185000F0B441EA012141EA014122F007047FF09E
:1018600000070023F0E80256083C85EA010586EAF5
:10187000010685FA47F5A3FA87F586FA47F6A5FA31
:1018800087F68EB9EED1F0BC01F0FF0102F007023D
:1018900032B110F8013B013A83EA010313B1F8D1E8
:1018A0000020704701387047002D06BF35460338C9
:1018B000073815F0010F07D1013015F4807F02BF02
:1018C000013015F4C03F0130F0BC0138704700BF53
:1018D000844641EA000313F003036DD1403A41D33B
:1018E00051F8043B40F8043B51F8043B40F8043BFA
:1018F00051F8043B40F8043B51F8043B40F8043BEA
:1019000051F8043B40F8043B51F8043B40F8043BD9
:1019100051F8043B40F8043B51F8043B40F8043BC9
:1019200051F8043B40F8043B51F8043B40F8043BB9
:1019300051F8043B40F8043B51F8043B40F8043BA9
:1019400051F8043B40F8043B51F8043B40F8043B99
:1019500051F8043B40F8043B51F8043B40F8043B89
:10196000403ABDD2303211D351F8043B40F8043B29
:1019700051F8043B40F8043B51F8043B40F8043B69
:1019800051F8043B40F8043B103AEDD20C3205D339
:1019900051F8043B40F8043B043AF9D2043208D031
:1019A000D2071CBF11F8013B00F8013B01D30B88A3
:1019B00003806046704700BF082A13D38B078DD081
:1019C00010F003038AD0C3F10403D21ADB071CBF53
:1019D00011F8013B00F8013B80D331F8023B20F8BD
:1019E000023B7BE7043AD9D3013A11F8013B00F8F6
:1019F000013BF9D20B7803704B7843708B7883707E
:101A0000604670478842F0B50DD98B1898420AD2CB
:101A10008118002A51D09A1A13F8014D01F8014D8E
:101A20009342F9D1F0BD0F2A48D941EA00039B0740
:101A300046D100F1100401F11003154653F8106C63
:101A400044F8106C53F80C6C44F80C6C53F8086CA8
:101A500044F8086C103D53F8046C44F8046C0F2DE6
:101A600003F1100304F11004E8D8A2F1100323F0ED
:101A70000F0302F00F0E1033BEF1030F194403449D
:101A800021D91E1F0D467446043C55F8047B46F8C8
:101A9000047F032CF8D8AEF1040424F003040434CA
:101AA0002344214402F0030262B1013B0A4411F8CD
:101AB000014B03F8014F8A42F9D1F0BD0346F3E729
:101AC0000346F2E7F0BD7246EEE700BFF9B1F8B5A4
:101AD00006461546B2B10C4600F032F8854201D8F0
:101AE0002046F8BD29463046FFF798F8074668B10A
:101AF0002A462146FFF7ECFE30462146FFF748F81C
:101B00003846F8BDFFF744F82846F8BDF8BD114641
:101B1000FFF784B870B50D46084C114606461A46C4
:101B200028460023236000F035F8431C00D070BD28
:101B30002368002BFBD0336070BD00BFBC010020C8
:101B400051F8040C0028BEBF091851F8043CC01815
:101B500004387047024B58221A604FF0FF3070472C
:101B6000BC010020024B58221A604FF0FF30704732
:101B7000BC010020024B58221A600020704700BFB1
:101B8000BC010020024B58221A604FF0FF30704712
:101B9000BC010020024B58221A604FF0FF30704702
:101BA000BC010020044A05491368002B08BF0B46FE
:101BB0001844106018467047A0000020C0010020A3
:101BC000024B58221A604FF0FF307047BC010020D2
:101BD00081F0004102E000BF83F0004330B54FEADE
:101BE00041044FEA430594EA050F08BF90EA020F4B
:101BF0001FBF54EA000C55EA020C7FEA645C7FEADE
:101C0000655C00F0E2804FEA5454D4EB5555B8BF00
:101C10006D420CDD2C4480EA020281EA030382EA71
:101C2000000083EA010180EA020281EA0303362D03
:101C300088BF30BD11F0004F4FEA01314FF4801CD6
:101C40004CEA113102D0404261EB410113F0004FE8
:101C50004FEA03334CEA133302D0524263EB43039F
:101C600094EA050F00F0A780A4F10104D5F1200E3D
:101C70000DDB02FA0EFC22FA05F2801841F1000198
:101C800003FA0EF2801843FA05F359410EE0A5F16C
:101C900020050EF1200E012A03FA0EFC28BF4CF09D
:101CA000020C43FA05F3C01851EBE37101F0004553
:101CB00007D54FF0000EDCF1000C7EEB00006EEB60
:101CC0000101B1F5801F1BD3B1F5001F0CD34908EA
:101CD0005FEA30004FEA3C0C04F101044FEA445241
:101CE00012F5800F80F09A80BCF1004F08BF5FEAC8
:101CF000500C50F1000041EB045141EA050130BDA8
:101D00005FEA4C0C404141EB010111F4801FA4F14A
:101D10000104E9D191F0000F04BF01460020B1FA9F
:101D200081F308BF2033A3F10B03B3F120020CDAD7
:101D30000C3208DD02F1140CC2F10C0201FA0CF0B5
:101D400021FA02F10CE002F11402D8BFC2F1200C1A
:101D500001FA02F120FA0CFCDCBF41EA0C019040D0
:101D6000E41AA2BF01EB0451294330BD6FEA040419
:101D70001F3C1CDA0C340EDC04F11404C4F1200204
:101D800020FA04F001FA02F340EA030021FA04F316
:101D900045EA030130BDC4F10C04C4F1200220FA6D
:101DA00002F001FA04F340EA0300294630BD21FAAB
:101DB00004F0294630BD94F0000F83F4801306BF71
:101DC00081F480110134013D4EE77FEA645C18BF65
:101DD0007FEA655C29D094EA050F08BF90EA020FFC
:101DE00005D054EA000C04BF1946104630BD91EAF4
:101DF000030F1EBF0021002030BD5FEA545C05D1F7
:101E00004000494128BF41F0004130BD14F5800435
:101E10003CBF01F5801130BD01F0004545F0FE41A9
:101E200041F470014FF0000030BD7FEA645C1ABFDE
:101E3000194610467FEA655C1CBF0B46024650EA15
:101E4000013406BF52EA033591EA030F41F4002141
:101E500030BD00BF90F0000F04BF0021704730B5C7
:101E60004FF4806404F132044FF000054FF000019C
:101E700050E700BF90F0000F04BF0021704730B55D
:101E80004FF4806404F1320410F0004548BF404232
:101E90004FF000013EE700BF42004FEAE2014FEA87
:101EA00031014FEA02701FBF12F07F4393F07F4F62
:101EB00081F06051704792F0000F14BF93F07F4F94
:101EC000704730B54FF4607401F0004521F00041D7
:101ED00020E700BF50EA010208BF704730B54FF05D
:101EE00000050AE050EA010208BF704730B511F062
:101EF000004502D5404261EB41014FF4806404F19A
:101F000032045FEA915C3FF4DCAE4FF003025FEA1B
:101F1000DC0C18BF03325FEADC0C18BF033202EBA3
:101F2000DC02C2F1200300FA03FC20FA02F001FAFD
:101F300003FE40EA0E0021FA02F11444C1E600BF9C
:101F400070B54FF0FF0C4CF4E06C1CEA11541DBF4F
:101F50001CEA135594EA0C0F95EA0C0F00F0DEF81A
:101F60002C4481EA030621EA4C5123EA4C5350EAFF
:101F7000013518BF52EA033541F4801143F4801350
:101F800038D0A0FB02CE4FF00005E1FB02E506F0E1
:101F90000042E0FB03E54FF00006E1FB03569CF036
:101FA000000F18BF4EF0010EA4F1FF04B6F5007F3C
:101FB00064F5407404D25FEA4E0E6D4146EB0606AE
:101FC00042EAC62141EA55514FEAC52040EA5E5037
:101FD0004FEACE2EB4F1FD0C88BFBCF5E06F1ED8E1
:101FE000BEF1004F08BF5FEA500E50F1000041EB18
:101FF000045170BD06F0004646EA010140EA0200C5
:1020000081EA0301B4EB5C04C2BFD4EB0C0541EAE6
:10201000045170BD41F480114FF0000E013C00F3FB
:10202000AB8014F1360FDEBF002001F0004170BD1F
:10203000C4F10004203C35DA0C341BDC04F1140438
:10204000C4F1200500FA05F320FA04F001FA05F2C4
:1020500040EA020001F0004221F0004110EBD37091
:1020600021FA04F642EB06015EEA430E08BF20EABD
:10207000D37070BDC4F10C04C4F1200500FA04F360
:1020800020FA05F001FA04F240EA020001F00041F2
:1020900010EBD37041F100015EEA430E08BF20EA65
:1020A000D37070BDC4F1200500FA05F24EEA020EAD
:1020B00020FA04F301FA05F243EA020321FA04F0DC
:1020C00001F0004121FA04F220EA020000EBD37093
:1020D0005EEA430E08BF20EAD37070BD94F0000F93
:1020E0000FD101F00046400041EB010111F4801FC7
:1020F00008BF013CF7D041EA060195F0000F18BF78
:10210000704703F00046520043EB030313F4801FB3
:1021100008BF013DF7D043EA0603704794EA0C0F6D
:102120000CEA135518BF95EA0C0F0CD050EA410683
:1021300018BF52EA4306D1D181EA030101F0004100
:102140004FF0000070BD50EA410606BF1046194628
:1021500052EA430619D094EA0C0F02D150EA013634
:1021600013D195EA0C0F05D152EA03361CBF104675
:1021700019460AD181EA030101F0004141F0FE4114
:1021800041F470014FF0000070BD41F0FE4141F498
:10219000780170BD70B54FF0FF0C4CF4E06C1CEA98
:1021A00011541DBF1CEA135594EA0C0F95EA0C0F4D
:1021B00000F0A7F8A4EB050481EA030E52EA033508
:1021C0004FEA013100F088804FEA03334FF0805529
:1021D00045EA131343EA12634FEA022245EA111556
:1021E00045EA10654FEA00260EF000419D4208BF07
:1021F000964244F1FD0404F5407402D25B084FEAB4
:102200003202B61A65EB03055B084FEA32024FF45F
:1022100080104FF4002CB6EB020E75EB030E22BFBC
:10222000B61A754640EA0C005B084FEA3202B6EB7C
:10223000020E75EB030E22BFB61A754640EA5C002B
:102240005B084FEA3202B6EB020E75EB030E22BFBB
:10225000B61A754640EA9C005B084FEA3202B6EBBC
:10226000020E75EB030E22BFB61A754640EADC007B
:1022700055EA060E18D04FEA051545EA16754FEADD
:1022800006164FEAC30343EA52734FEAC2025FEAFB
:102290001C1CC0D111F4801F0BD141EA00014FF08A
:1022A00000004FF0004CB6E711F4801F04BF01435B
:1022B0000020B4F1FD0C88BFBCF5E06F3FF6AFAE77
:1022C000B5EB030C04BFB6EB020C5FEA500C50F107
:1022D000000041EB045170BD0EF0004E4EEA11318A
:1022E00014EB5C04C2BFD4EB0C0541EA045170BD91
:1022F00041F480114FF0000E013C90E645EA060ED5
:102300008DE60CEA135594EA0C0F08BF95EA0C0F02
:102310003FF43BAF94EA0C0F0AD150EA01347FF44A
:1023200034AF95EA0C0F7FF425AF104619462CE721
:1023300095EA0C0F06D152EA03353FF4FDAE104684
:10234000194622E750EA410618BF52EA43067FF4D5
:10235000C5AE50EA41047FF40DAF52EA43057FF465
:10236000EBAE12E74FEA4102B2F1E04324BFB3F50E
:10237000001CDCF1FE5C0DD901F0004C4FEAC002FC
:102380004CEA5070B2F1004F40EB830008BF20F0E0
:102390000100704711F0804F21D113F13872BCBF9A
:1023A00001F00040704741F480114FEA5252C2F1EF
:1023B0001802C2F1200C10FA0CF320FA02F018BF38
:1023C00040F001004FEAC1234FEAD32303FA0CFC8B
:1023D00040EA0C0023FA02F34FEA4303CCE77FEA1A
:1023E000625307D150EA01331EBF4FF0FE4040F464
:1023F0004000704701F0004040F0FE4040F4000013
:10240000704700BF53B94AB9002908BF00281CBF54
:102410004FF0FF314FF0FF3000F07EB9ADF1080C06
:102420006DE904CE00F006F8DDF804E0DDE90223F2
:1024300004B070472DE9F0478C460E460446089DCF
:10244000002B50D18A4217466CD9B2FA82FEBEF1F7
:10245000000F0BD0CEF1200420FA04F401FA0EF69E
:1024600044EA060C02FA0EF700FA0EF44FEA174996
:10247000220CBCFBF9F01FFA87F809FB10C642EAF0
:10248000064600FB08F3B34209D9F61900F1FF3202
:1024900080F02281B34240F21F8102383E44F61A96
:1024A000A2B2B6FBF9F309FB136642EA064403FB4A
:1024B00008F8A04509D9E41903F1FF3280F00A8138
:1024C000A04540F20781023B3C44C8EB040443EAC8
:1024D00000400021002D62D024FA0EF400232C606D
:1024E0006B60BDE8F0878B4207D9002D55D00021E5
:1024F00085E841000846BDE8F087B3FA83F100297A
:1025000040F09080B34202D3824200F2F880841AF5
:1025100066EB03060120B446002D40D085E810107C
:10252000BDE8F08712B90127B7FBF2F7B7FA87FECB
:10253000BEF1000F35D1F31B4FEA17481FFA87FC95
:102540000121B3FBF8F0220C08FB103642EA0646E4
:102550000CFB00F3B34207D9F61900F1FF3202D2A7
:10256000B34200F2CE801046F61AA2B2B6FBF8F3E0
:1025700008FB136642EA06440CFB03FCA44507D99A
:10258000E41903F1FF3202D2A44500F2B5801346EC
:10259000CCEB040443EA00409CE729462846BDE80A
:1025A000F087CEF1200106FA0EF307FA0EF720FAB3
:1025B00001F94FEA1748CE4049EA0309B6FBF8FA99
:1025C0004FEA194408FB1A661FFA87FC44EA0643DF
:1025D0000AFB0CF29A4200FA0EF40AD9DB190AF14E
:1025E000FF3180F087809A4240F28480AAF1020A8B
:1025F0003B449B1A1FFA89F9B3FBF8F108FB11332E
:1026000049EA034301FB0CF69E4207D9DB1901F1AD
:10261000FF326BD29E4269D902393B449B1B41EA8F
:102620000A418EE7C1F1200E22FA0EF48B402343BB
:1026300020FA0EF706FA01F44FEA134C26FA0EF6CA
:102640003C43B6FBFCF9270C0CFB19661FFA83F818
:1026500047EA064609FB08F7B74202FA01F200FA18
:1026600001FA08D9F61809F1FF3041D2B7423FD933
:10267000A9F102091E44F61BA0B2B6FBFCF40CFB48
:10268000146640EA064704FB08F8B84507D9FF1866
:1026900004F1FF3028D2B84526D9023C1F4444EA51
:1026A0000940C8EB0707A0FB02894F4544464E4648
:1026B00014D329D065B3BAEB040367EB060707FA16
:1026C0000EFECB40CF404EEA030385E88800002190
:1026D000BDE8F0871346F8E61046E0E6B8EB0204E2
:1026E00069EB03060138E5E70446D8E7114695E7AC
:1026F0008146C0E78A467CE7023B3C4448E70846FF
:102700000AE702383E442FE7C245E7D33E46D1E709
:102710002946BDE8F08700BF704700BF30B595B0CF
:102720003022002108A8FDF7ADFD00240394049495
:1027300005940694079401941A4B1A6C42F0805247
:102740001A641B6C03F080530193019B0294164B97
:102750001A6842F480421A601B6803F480430293B3
:10276000029B0225089501230B9310230C930E95D1
:102770000F94082310934823119312950323139366
:1027800008A801F0EDF80F230393049505944FF486
:10279000805306930794294603A801F011FB15B056
:1027A00030BD00BF003802400070004008B501F0A5
:1027B00065FDFFF7B3FF00F0FDF800F03BFA00F015
:1027C00005FA00F01DFA00F099F9674C204600F078
:1027D000FFFB3221204600F095FC204600F0B8FDBA
:1027E00010F4007F00F08380204600F0E7FC80B208
:1027F0005E4C208007EE900AF8EEE77A9FED5C8A47
:1028000067EE887ADFED5B8A67EEA87A17EE900AAA
:10281000FFF742FB02460B465748FDF797FD23881A
:1028200007EE903AF8EEE77A67EE887A27EEA88A04
:10283000524B83ED008A524BD3ED008AB4EEE88A06
:10284000F1EE10FA25DD4F4BD3ED007A77EEE87A02
:1028500017EE900AFFF720FB02460B4600204A497C
:10286000FFF798FC04460D4678EE687A17EE900A5A
:10287000FFF712FB22462B46FFF762FB02460B4690
:1028800000204249FFF7A8F9FFF76CFD404B1860A4
:1028900024E0404BD3ED007A78EEE77A17EE900A09
:1028A000FFF7FAFA02460B4600203749FFF772FCA1
:1028B00004460D4678EE687A17EE900AFFF7ECFAB8
:1028C00022462B46FFF73CFB02460B4600202F49D1
:1028D000FFF782F9FFF746FD2D4B18602C4B186867
:1028E000FFF7DAFA02460B462B48FDF72FFD42F2BE
:1028F000107001F0EFFC264B93ED007AF3EE097AAD
:10290000B4EEE77AF1EE10FA3FF65FAF234C002207
:102910004FF40051204601F009FC2148FDF7A0FDCD
:1029200000224FF48051204601F000FC1D48FDF7C5
:1029300097FD4FF4FA7001F0CDFC01224FF4805165
:10294000204601F0F3FB1848FDF78AFD4FF47A703A
:1029500001F0C0FC01224FF40051204601F0E6FBDB
:102960001248FDF77DFD30E7B0000020A4000020F4
:10297000333353400000803918440008A800002079
:1029800068000020640000200000084000001C4097
:10299000AC0000206C0000202C4400080000024025
:1029A0003C440008484400085444000860440008BF
:1029B000704700BF2DE9F0478AB0002405940694C3
:1029C0000794089409940094464B1A6B42F0010254
:1029D0001A631A6B02F001020092009A01941A6BBA
:1029E00042F010021A631A6B02F010020192019A6F
:1029F00002941A6B42F002021A631A6B02F002028E
:102A00000292029A03941A6B42F008021A631A6B3C
:102A100002F008020392039A04941A6B42F0040233
:102A20001A631B6B03F004030493049BDFF8C0A03C
:102A300022464FF47841504601F078FBDFF8B4901D
:102A400022464FF44041484601F070FBDFF8A88071
:102A500022464FF47C41404601F068FB224F22465B
:102A60004FF40071384601F061FB204E22464FF4CE
:102A70007C51304601F05AFB4FF478430593012511
:102A800006950794089405A9504601F06FFA4FF493
:102A90004043059306950794089405A9484601F01C
:102AA00065FA4FF47C43059306950794089405A9AD
:102AB000404601F05BFA4FF40073059306950794C6
:102AC000089405A9384601F051FA4FF47C53059358
:102AD00006950794089405A9304601F047FA0AB014
:102AE000BDE8F087003802400008024000000240C4
:102AF0000010024000040240000C024000B585B006
:102B0000002300930193029303931348134A026036
:102B1000436083600361037680F82030C362104A0B
:102B20008262C3600122C26180F83030426100F0ED
:102B300025FA08B1FFF73CFF04230093012301931A
:102B4000002302936946044800F03CFB08B1FFF7FC
:102B50002FFF05B05DF804FBB0000020002001400D
:102B60000100000F00B589B000230393049305937F
:102B700006930793026803F1804303F590339A426A
:102B80001ED10021019103F58C335A6C42F48072FE
:102B90005A645A6C02F480720192019A02911A6B83
:102BA00042F001021A631B6B03F001030293029BC4
:102BB000102303930323049303A9034801F0D6F9D8
:102BC00009B05DF804FB00BF0000024008B50A48E8
:102BD0000A4B03604FF4E133436000238360C3601A
:102BE00003610C2242618361C36100F08DFD08B175
:102BF000FFF7DEFE08BD00BF38010020004C00409A
:102C000008B50A480A4B03604FF4E13343600023E0
:102C10008360C36003610C2242618361C36100F081
:102C200073FD08B1FFF7C4FE08BD00BFF800002027
:102C30000010014008B50A480A4B03604FF41643E0
:102C4000436000238360C36003610C22426183619F
:102C5000C36100F059FD08B1FFF7AAFE08BD00BF2F
:102C6000780100200044004010B58CB00023079389
:102C7000089309930A930B930368494A93422DD111
:102C800000240194474B1A6C42F400221A641A6C17
:102C900002F400220192019A02941A6B42F004029B
:102CA0001A631B6B03F004030293029B4FF440630F
:102CB0000793022308930123099303230A9308230C
:102CC0000B9307A9384801F051F9224621463420D8
:102CD00001F058FA342001F087FA5EE0334A93425B
:102CE0002CD1002403942F4B5A6C42F010025A64EA
:102CF0005A6C02F010020392039A04941A6B42F089
:102D000002021A631B6B03F002030493049BC023AB
:102D10000793022308930123099303230A930723AC
:102D20000B9307A9224801F021F9224621462520CC
:102D300001F028FA252001F057FA2EE01D4A9342AF
:102D40002BD100240594174B1A6C42F400321A64FC
:102D50001A6C02F400320592059A06941A6B42F03E
:102D600008021A631B6B03F008030693069B60239B
:102D70000793022308930123099303230A9307234C
:102D80000B9307A90C4801F0F1F8224621462620B2
:102D900001F0F8F9262001F027FA0CB010BD00BFB1
:102DA000004C004000380240000802400010014082
:102DB0000004024000440040000C0240704700BF85
:102DC000FEE700BFFEE700BFFEE700BFFEE700BF73
:102DD000704700BF704700BF704700BF08B501F0E3
:102DE00067FA08BD08B5024800F024FD08BD00BF21
:102DF000F800002008B5024800F01CFD08BD00BF27
:102E00007801002008B5024800F014FD08BD00BF9D
:102E10003801002082B0002100910B4B5A6C42F423
:102E200080425A645A6C02F480420092009A0191E6
:102E30001A6C42F080521A641B6C03F080530193A9
:102E4000019B02B0704700BF00380240494B5A68EE
:102E500022F440325A60596842680A435A60026854
:102E6000536823F48073536002685368016943EA2E
:102E7000012353600268536823F040735360026873
:102E8000516883680B4353600268936823F40063BE
:102E9000936002689168C3680B439360826A364B03
:102EA0009A4214D00268936823F0706393600268BA
:102EB0009168836A0B4393600268936823F04053E0
:102EC000936002689168C36A0B43936009E00268EB
:102ED000936823F0706393600268936823F0405313
:102EE00093600268936823F002039360026893681A
:102EF000017E43EA4103936090F820308BB1026871
:102F0000536843F4006353600268536823F46043DA
:102F1000536001684A68436A013B42EA43334B60AD
:102F200004E00268536823F4006353600268D36AC4
:102F300023F47003D3620168CA6AC369013B42EAA1
:102F40000353CB620268936823F4007393600268B2
:102F5000936890F8301043EA4123936002689368C5
:102F600023F48063936002689368416943EA812394
:102F700093607047002301400100000F30B310B58B
:102F80000446036C2BB9FFF7EDFD0023636484F85E
:102F90003C30236C13F0100F13D1236C23F48853AF
:102FA00023F0020343F0020323642046FFF74EFFA1
:102FB00000206064236C23F0030343F001032364C7
:102FC00000E00120002384F83C3010BD0120704750
:102FD00082B00023019390F83C30012B78D001237C
:102FE00080F83C3003689A6812F0010F13D19A6898
:102FF00042F001029A603E4B1B683E4AA2FB03234B
:103000009B0C03EB4303019302E0019B013B019303
:10301000019B002BF9D10268936813F0010F59D07E
:10302000036C23F4E06323F0010343F4807303642F
:10303000536813F4806F05D0036C23F4405343F4BA
:1030400080530364036C13F4805F04D0436C23F05B
:103050000603436401E000234364002380F83C300E
:103060006FF022031360244B5B6813F01F0F21D114
:103070000368224A934213D002F58072934205D12D
:1030800002F50072526812F01F0F09D01C4A9342D9
:1030900022D102F58072526802F01F020F2A1DD859
:1030A0009A6812F0405F1BD19A6842F080429A60A1
:1030B00000201AE00368114A934213D19A6812F073
:1030C000405F11D19A6842F080429A6000200CE083
:1030D00002200AE0002008E0002006E0002004E0D2
:1030E000002002E0002000E0002002B0704700BF96
:1030F0007800002083DE1B430023014000200140B4
:103100000022014070B503689A6812F4806F0CD0F9
:103110009B6813F4807F08D0036C43F020030364A2
:10312000002380F83C30012070BD0D46044601F0BC
:10313000CBF8064611E0B5F1FF3F0ED025B101F006
:10314000C3F8801B854208D2236C43F00403236438
:10315000002384F83C30032070BD23681A6812F005
:10316000020FE8D06FF012021A60236C43F4007370
:10317000236423689A6812F0405F17D1227EBAB99F
:10318000DA6A12F4700F03D09B6813F4806F11D1C8
:10319000236C23F480732364236C13F4805F0BD1BE
:1031A000236C43F001032364002070BD002070BD38
:1031B000002070BD002070BD002070BD0368D86C79
:1031C000704700BF30B482B00023019390F83C30C8
:1031D000012B00F0B280012380F83C300B68092BF2
:1031E00017D90568EA689BB203EB43031E3B07242B
:1031F00004FA03F322EA0303EB600468E5688A68D3
:103200000B8803EB43031E3B02FA03F32B43E360FB
:1032100013E005682A699BB203EB4303072404FA11
:1032200003F322EA03032B61046825698B680A888B
:1032300002EB420293402B4323614B68062B16D8C6
:1032400005686A6B03EB8303053B1F2404FA03F351
:1032500022EA03036B630468656B4B6803EB83032B
:10326000053B0A8802FA03F32B4363632EE00C2B21
:1032700016D805682A6B03EB8303233B1F2404FA4B
:1032800003F322EA03032B630468256B4B6803EB0B
:103290008303233B0A8802FA03F32B43236315E0DD
:1032A0000568EA6A03EB8303413B1F2404FA03F336
:1032B00022EA0303EB620468E56A4B6803EB8303CD
:1032C000413B0A8802FA03F32B43E36202681D4B79
:1032D0009A4207D10B68122B04D11B4A536843F45E
:1032E000800353600268174B9A4221D10B68103B50
:1032F000012B1DD8144A536843F4000353600B6834
:10330000102B15D1114B1B6802F1467202F52E32BB
:1033100002F28332A2FB03239B0C03EB83035A00CC
:10332000019202E0019B013B0193019B002BF9D12B
:10333000002380F83C30184600E0022002B030BC88
:10334000704700BF002001400023014078000020AA
:10335000006C70470268D36823F49073D3600268EE
:10336000536923F001035361202380F83A307047FA
:1033700090F83930DBB2212B2BD18368B3F5805F15
:103380000FD1036A02681B88C3F308035360036903
:103390001BB9036A0233036209E0036A0133036263
:1033A00005E00268036A591C01621B785360C38CF4
:1033B0009BB2013B9BB2C3846BB90268D36823F014
:1033C0008003D3600268D36843F04003D3600020D9
:1033D0007047022070470020704700BF2DE9F84376
:1033E000044601680B6923F44052C36813430B6120
:1033F00081680369194343691943C3691943006824
:10340000C26822F4164323F00C030B43C360216807
:103410004B6923F44072A36913434B61E369B3F52D
:10342000004F40F0BB80276803F1804303F5104351
:103430009F4203D003F580639F4257D100F086FD81
:1034400000EB800000EB800065686D00B0FBF5F5D7
:10345000AB4EA6FB05356D092D0100F077FD00EBA5
:10346000800000EB800063685B00B0FBF3F900F0C4
:103470006DFD00EB800000EB800063685B00B0FB3B
:10348000F3F3A6FB03235B094FF0640808FB1393D7
:10349000DB003233A6FB03235B095B0003F4F87304
:1034A0001D4400F053FD00EB800000EB80006368DA
:1034B0005B00B0FBF3F900F049FD00EB800000EB8E
:1034C000800063685B00B0FBF3F3A6FB03235B099A
:1034D00008FB13984FEAC80808F13208A6FB083623
:1034E000C6F342163544BD60BDE8F88300F01EFD0A
:1034F00000EB800000EB800065686D00B0FBF5F527
:103500007F4EA6FB05356D092D0100F00FFD00EB88
:10351000800000EB800063685B00B0FBF3F900F013
:1035200005FD00EB800000EB800063685B00B0FBF2
:10353000F3F3A6FB03235B094FF0640808FB139326
:10354000DB003233A6FB03235B095B0003F4F87353
:103550001D4400F0EBFC00EB800000EB8000636892
:103560005B00B0FBF3F900F0E1FC00EB800000EB46
:10357000800063685B00B0FBF3F3A6FB03235B09E9
:1035800008FB13984FEAC80808F13208A6FB083672
:10359000C6F342163544BD60BDE8F8832668594B32
:1035A0009E4203D003F580639E4254D100F0CEFCCE
:1035B00000EB800000EB80006568AD00B0FBF5F526
:1035C0004F4FA7FB05356D092D0100F0BFFC00EB47
:1035D000800000EB800063689B00B0FBF3F800F014
:1035E000B5FC00EB800000EB800063689B00B0FB43
:1035F000F3F3A7FB03235B094FF0640909FB138373
:103600001B013233A7FB03235B0903F0F0031D44C6
:1036100000F09CFC00EB800000EB800063689B00E6
:10362000B0FBF3F800F092FC00EB800000EB8000B0
:1036300063689B00B0FBF3F3A7FB03235B0909FB63
:1036400013831B013233A7FB0323C3F343131D442E
:10365000B560BDE8F88300F069FC00EB800000EB8A
:1036600080006568AD00B0FBF5F5254FA7FB05357B
:103670006D092D0100F05AFC00EB800000EB80008A
:1036800063689B00B0FBF3F800F050FC00EB800097
:1036900000EB800063689B00B0FBF3F3A7FB032300
:1036A0005B094FF0640909FB13831B013233A7FB4D
:1036B00003235B0903F0F0031D4400F037FC00EB2B
:1036C000800000EB800063689B00B0FBF3F800F023
:1036D0002DFC00EB800000EB800063689B00B0FBDA
:1036E000F3F3A7FB03235B0909FB13831B013233AD
:1036F000A7FB0323C3F343131D44B560BDE8F88360
:103700001F85EB510010014068B310B5044690F8D6
:10371000393013F0FF0F04D1002380F83830FFF761
:10372000A3FA242384F839302268D36823F40053A1
:10373000D3602046FFF752FE2268136923F49043BA
:1037400013612268536923F02A0353612268D36806
:1037500043F40053D3600020E063202384F8393021
:1037600084F83A3010BD0120704700BF704700BF99
:1037700008B50168CB6823F04003CB60202380F8B4
:103780003930FFF7F3FF002008BD00BF704700BFCE
:1037900008B590F83A30DBB2222B44D18368B3F5F8
:1037A000805F13D1826A036943B903685B68C3F31E
:1037B00008031380836A0233836218E003685B683E
:1037C000DBB21380836A0133836210E0036933B98B
:1037D000836A5A1C8262026852681A7007E0826A21
:1037E000531C836203685B6803F07F031370C38D0F
:1037F0009BB2013B9BB2C385BBB90268D36823F07F
:103800002003D3600268D36823F48073D360026816
:10381000536923F001035361202380F83A30FFF706
:10382000B5FF002008BD022008BD002008BD00BF74
:10383000704700BF10B5044602681368D16852692A
:1038400013F00F0009D113F0200F06D011F0200F54
:1038500003D02046FFF79CFF10BD002862D012F075
:10386000010202D111F4907F5CD013F0010F06D059
:1038700011F4807F03D0E06B40F00100E06313F0AF
:10388000040F04D01AB1E06B40F00200E06313F0C3
:10389000020F04D01AB1E06B40F00400E06313F0B3
:1038A000080F04D01AB1E26B42F00802E263E26B47
:1038B000002A4AD013F0200F05D011F0200F02D0BB
:1038C0002046FFF765FF23685B6903F04003E26B66
:1038D00012F0080F00D1FBB12046FFF73BFD236833
:1038E0005A6912F0400F13D05A6922F040025A610F
:1038F000636B4BB1154A1A65606B00F01DFC20B379
:10390000606B036D984710BD2046FFF791FF10BD17
:103910002046FFF78DFF10BD2046FFF789FF0023EB
:10392000E36310BD13F0800F06D011F0800F03D0B9
:103930002046FFF71DFD10BD13F0400F05D011F01C
:10394000400F02D02046FFF713FF10BD5139000889
:1039500008B5806B0023C385C384FFF769FF08BDEA
:10396000002800F0B58170B582B00446036813F0FA
:10397000010F5AD0A04B9B6803F00C03042B0AD014
:103980009D4B9B6803F00C03082B0DD19A4B5B6891
:1039900013F4800F08D0984B1B6813F4003F44D0F9
:1039A0006368002B41D195E16368B3F5803F05D191
:1039B000914A136843F48033136015E0B3F5A02FE8
:1039C00009D18D4B1A6842F480221A601A6842F4B9
:1039D00080321A6008E0884B1A6822F480321A603C
:1039E0001A6822F480221A6063687BB100F06CFCD4
:1039F000054605E000F068FC401B642800F26C817D
:103A00007D4B1B6813F4003FF4D00EE000F05CFC2B
:103A1000054605E000F058FC401B642800F25E817A
:103A2000754B1B6813F4003FF4D1236813F0020FA9
:103A300050D0714B9B6813F00C0F0AD06E4B9B68F3
:103A400003F00C03082B16D16B4B5B6813F4800F4B
:103A500011D1694B1B6813F0020F03D0E368012BEF
:103A600040F03E81644A136823F0F803216943EA79
:103A7000C10313602EE0E368D3B101225F4B1A60EB
:103A800000F022FC054605E000F01EFC401B022869
:103A900000F22881584B1B6813F0020FF4D0564AED
:103AA000136823F0F803216943EAC103136011E0AE
:103AB0000022524B1A6000F007FC054605E000F0BA
:103AC00003FC401B022800F20F814B4B1B6813F0D4
:103AD000020FF4D1236813F0080F26D0636993B165
:103AE0000122474B1A6000F0EFFB054605E000F0AD
:103AF000EBFB401B022800F2F9803F4B5B6F13F099
:103B0000020FF4D011E000223D4B1A6000F0DCFB04
:103B1000054605E000F0D8FB401B022800F2E880D3
:103B2000354B5B6F13F0020FF4D1236813F0040FD1
:103B30007CD0314B1B6C13F0805F0DD100230193BF
:103B40002D4B1A6C42F080521A641B6C03F08053A8
:103B50000193019B012500E000252A4B1B6813F40B
:103B6000807F13D1274A136843F48073136000F0F9
:103B7000ABFB064605E000F0A7FB801B022800F225
:103B8000B980204B1B6813F4807FF4D0A368012B0D
:103B900005D1194A136F43F00103136714E0052B95
:103BA00009D1154B1A6F42F004021A671A6F42F0DE
:103BB00001021A6708E0104B1A6F22F001021A671F
:103BC0001A6F22F004021A67A3688BB100F07CFB25
:103BD000064607E000F078FB801B41F288339842EC
:103BE00000F28A80044B1B6F13F0020FF2D017E033
:103BF00000F06AFB06460EE0003802400000474233
:103C0000800E47420070004000F05EFB801B41F2D6
:103C10008833984272D8404B1B6F13F0020FF3D1D8
:103C200025B13D4A136C23F080531364A369002B24
:103C300066D0394A926802F00C02082A62D0022B40
:103C400033D10022354B1A6000F03EFB054604E0FC
:103C500000F03AFB401B022856D82F4B1B6813F08C
:103C6000007FF5D1E269236A1343626A43EA821353
:103C7000A26A5208013A43EA0243E26A43EA026353
:103C8000254A53600122254B1A6000F01DFB0446B3
:103C900004E000F019FB001B022837D81E4B1B68FC
:103CA00013F0007FF5D0002033E000221B4B1A6098
:103CB00000F00AFB044604E000F006FB001B0228AB
:103CC00026D8154B1B6813F0007FF5D1002020E0AB
:103CD0000120704701201CE003201AE0032018E0B7
:103CE000012016E0032014E0032012E0032010E07E
:103CF00003200EE003200CE003200AE0032008E08C
:103D0000002006E0012004E0032002E0032000E0A0
:103D1000032002B070BD00BF00380240600047427F
:103D200038B5244B9B6803F00C03042B3FD0082BC1
:103D300001D0214838BD1F4B5A6802F03F025B6832
:103D400013F4800F0AD01B4B5968C1F3881100236C
:103D50001A48A1FB0001FEF755FB1FE0154B5B68FD
:103D6000C3F38813DC000025690141EAD4616001D6
:103D7000041B61EB0505A90141EA9461A001001B48
:103D800061EB0501C01841F100018B0243EA905339
:103D90008402204619460023FEF734FB054B5B687E
:103DA000C3F3014301335B00B0FBF3F038BD0348BC
:103DB00038BD00BF003802400024F40040787D0187
:103DC000002800F0978070B50446514B1B6803F043
:103DD0000F038B4208D2CBB24D4A1370136803F025
:103DE0000F03994240F08880236813F0020F17D028
:103DF00013F0040F04D0474A936843F4E0539360F0
:103E0000236813F0080F04D0424A936843F46043D8
:103E100093604048836823F0F002A36813438360F3
:103E20000D46236813F0010F2FD06268012A05D1D7
:103E3000384B1B6813F4003F0ED15FE0931E012B3B
:103E400005D8344B1B6813F0007F05D158E0314B87
:103E50001B6813F0020F55D02E498B6823F0030323
:103E600013438B6000F030FA064606E000F02CFAAF
:103E7000801B41F28833984246D8264B9B6803F05A
:103E80000C036268B3EB820FF0D1214B1B6803F087
:103E90000F039D4207D2EAB21D4B1A701B6803F054
:103EA0000F039D4232D1236813F0040F06D0194945
:103EB0008B6823F4E052E36813438B60236813F0AC
:103EC000080F07D0134A936823F46043216943EA3B
:103ED000C1039360FFF724FF0E4B9B68C3F30313EA
:103EE0000D4AD35CD8400D4B1860002000F0A0F9BB
:103EF000002070BD01207047012070BD012070BD01
:103F0000012070BD012070BD032070BD012070BD77
:103F1000003C0240003802406C4400087800002059
:103F2000014B1868704700BF7800002008B5FFF704
:103F3000F7FF044B9B68C3F38223034AD35CD8404A
:103F400008BD00BF003802407C44000808B5FFF7F8
:103F5000E7FF044B9B68C3F34233034AD35CD8406A
:103F600008BD00BF003802407C440008F0B583B0B3
:103F70000024CDE00123A3400A6803EA0205AB4216
:103F800040F0C5804A68022A01D0122A10D1E60802
:103F9000083650F826C004F0070297000F22BA40F6
:103FA0002CEA020E0A69BA404EEA020240F82620C4
:103FB000026867000326BE40F64302EA060E4A681E
:103FC00002F00302BA404EEA020202604A6802F1BD
:103FD000FF3EBEF1010F03D9112A01D0122A10D1E0
:103FE000826806EA020ECA68BA404EEA020282609D
:103FF000426822EA03034A68C2F30012A2401A434D
:104000004260C3681E408B68BB403343C3604B684B
:1040100013F0805F7BD000230193404B5A6C42F435
:1040200080425A645B6C03F480430193019BA608B1
:10403000B21C3B4B53F8227004F003039B000F2289
:104040009A4027EA0207374A90421DD002F5806263
:1040500090421BD002F58062904219D002F5806236
:10406000904217D002F58062904215D002F580622E
:10407000904213D002F58062904211D002F5806226
:1040800090420FD107220EE000220CE001220AE04C
:10409000022208E0032206E0042204E0052202E0F6
:1040A000062200E0082202FA03F33B4302361C4AD0
:1040B00042F826301C4B1A68EB4302EA03064F68AD
:1040C00017F4803F01D045EA0206174A166052688D
:1040D00003EA02064F6817F4003F01D045EA0206E2
:1040E000114A5660926803EA02064F6817F4801F6F
:1040F00001D045EA02060C4A9660D26813404E6829
:1041000016F4001F01D045EA0203074AD3600134C8
:104110000F2C7FF62FAF03B0F0BD00BF0038024078
:104120000038014000000240003C01400AB18161BA
:10413000704709048161704790F83530DBB2022B7B
:1041400003D08023436501207047052380F8353074
:104150000268136823F0010313600020704700BF5A
:10416000074AD36823F4E0631B041B0C000200F42D
:10417000E060184340F0BF6040F40030D06070470A
:1041800000ED00E030B4164BDB68C3F30223C3F14B
:104190000704042C28BF04241D1D062D01D9DD1E93
:1041A00000E00025012303FA04F4013C2140A9406A
:1041B000AB40013B1A400A43002808DB1201D2B28F
:1041C00000F1604000F5614080F8002305E000F058
:1041D0000F001201D2B2034B1A5430BC704700BF1B
:1041E00000ED00E014ED00E0002808DB420900F0DB
:1041F0001F00012303FA00F0014B43F8220070472F
:1042000000E100E00138B0F1807F0AD2064B58602F
:10421000F021064A82F823100020986007221A60D5
:1042200070470120704700BF10E000E000ED00E0A3
:1042300010B504460E4B18784FF47A73B3FBF0F3C5
:104240000C4A1068B0FBF3F0FFF7DCFF58B90F2CF5
:104250000BD8002221464FF0FF30FFF793FF064BAB
:104260001C60002010BD012010BD012010BD00BF4A
:1042700074000020780000207000002008B50B4B6F
:104280001A6842F400721A601A6842F480621A6076
:104290001A6842F480721A600320FFF761FF002061
:1042A000FFF7C6FFFEF7B6FD002008BD003C024048
:1042B000034A1368034909780B441360704700BF31
:1042C000B801002074000020014B1868704700BF3F
:1042D000B801002038B50446FFF7F6FF0546B4F1F3
:1042E000FF3F02D0044B1B781C44FFF7EDFF401B3F
:1042F0008442FAD838BD00BF740000200E49D1F8BE
:10430000883043F47003C1F888300C4B1A6842F0CF
:1043100001021A60002098601A6822F0847222F468
:1043200080321A60064A5A601A6822F480221A60A3
:10433000D860044B8B60704700ED00E0003802400D
:104340001030002400000108DFF834D0002103E021
:104350000C4B5B58435004310B480C4B42189A42AB
:10436000F6D30B4A02E0002342F8043B094B9A4281
:10437000F9D3FFF7C3FFFBF75DFFFEF717FA7047AE
:1043800000000220D4440008000000207C0000202F
:104390007C000020C0010020FEE70000F8B500BF4F
:1043A000F8BC08BC9E467047F8B500BFF8BC08BC16
:0443B0009E4670476E
:1043B40004000020000000000000000000000000D5
:1043C40000000000000000000000000000000000E9
:1043D40000000000000000000000000000000000D9
:1043E40000000000000000000000000000000000C9
:1043F40000000000000000000000000000000000B9
:1044040000000000000000000000000000000000A8
:1044140000000000766F6C74616765203A202531D6
:104424002E3366560A0000004D345F50483A20256A
:10443400312E31660A00000072656C6179313A31BF
:104444000000000072656C6179323A3100000000AE
:1044540072656C6179323A300000000072656C61FB
:1044640079313A3000000000000000000000000034
:104474000102030406070809000000000102030406
:1044840043000000232D302B20000000686C4C00FA
:104494006566674546470000303132333435363778
:1044A400383941424344454600000000303132333C
:1044B400343536373839616263646566000000005C
:0844C40070DFFF7F0100000022
:0444CC00FD010008E6
:0444D000D50100080A
:1044D4000400002000000000F8430008D84300084E
:1044E400B8430008000000000000000000000000C5
:1044F40000000000844400080000000000000000E8
:1045040000000000000000000000000000000000A7
:104514000000000000000000000000000000000097
:104524000000000000000000000000000000000087
:104534000000000085EB01400000C03F9A99793FDC
:0C45440010000000010000000024F40042
:040000050800434963
:00000001FF
